:100000000C947E000C949B000C949B000C949B0021
:100010000C949B000C949B000C949B000C949B00F4
:100020000C949B000C94B6070C940E070C94990743
:100030000C945F070C947C070C94F1060C94420717
:100040000C94AA060C949B000C948F080C949B00B3
:100050000C9463090C943E020C949B000C949B003E
:100060000C949B000C949B000C949B000C949B00A4
:100070000C949B000C949B000C9480080C949B00A7
:100080000C9454090C949B000C949B00084AD73B99
:100090003BCE016E84BCBFFDC12F3D6C74319ABD57
:1000A00056833DDA3D00C77F11BED9E4BB4C3E917B
:1000B0006BAAAABE000000803F66693A25642E251F
:1000C0006420202B2D2025642E2564200D0A00306D
:1000D00031323334353637383941424344454600AE
:1000E00000000100080040000001000400000100C1
:1000F00008002000400080000001000411241FBE01
:10010000CFEFD0E1DEBFCDBF12E0A0E0B1E0E8EF7D
:10011000F8E202C005900D92A830B107D9F713E0BC
:10012000A8E0B2E001C01D92A337B107E1F70E9439
:100130009D000C947A140C9400002F923F924F92E1
:100140005F926F927F928F929F92AF92BF92CF9267
:10015000DF92EF92FF920F931F93DF93CF93CDB770
:10016000DEB7C650D1400FB6F894DEBF0FBECDBF8C
:100170000E945B0A40E855E260E070E080E00E9487
:10018000DE078EE298E00E94F7020E94E8040E94D7
:10019000F6011ABA1BBA87E00E94090280E00E94A9
:1001A0000E02882499249E012F5F3E4FCB5FDE4FC5
:1001B00039832883C550D14037C080E00E94230294
:1001C0007C0181E00E942302A0E0B0E0BC01CD01EF
:1001D0000E94B90E20E030E84FEF53E40E94D50BA7
:1001E0005B016C0100E010E0C801B7010E94B90E8C
:1001F00020E030E84FEF53E40E94D50BA6019501B3
:100200000E94D611F401EE0FFF1FEE0FFF1F21E039
:1002100030E02C0F3D1FE20FF31F60837183828358
:1002200093830894811C911C30E48316910428F276
:100230006E010894C11CD11C460160E070E080E0B2
:1002400090E0F40121913191419151914F010E942F
:10025000060CCB5FDE4F28813981C550D140821614
:10026000930679F720E030E040E85CE30E94330C2D
:100270002BED3FE049E450E40E94060C20E030E022
:1002800044E353E40E94330C2BED3FE049E450E497
:100290000E942D0DCF5FDE4F688379838A839B8315
:1002A000C150D1400F2EF0E0EF2EF0E0FF2EF0E035
:1002B0000F2FF0E01F2FF02DCF5FDE4F2881398107
:1002C0004A815B81C150D140F60161917191819168
:1002D00091916F010E94D50B9B01AC010E94330CE0
:1002E0009B01AC01C801B7010E94060C7B018C0187
:1002F000C814D90409F720E030E04CE752E40E942A
:100300002D0D0E94C61320E030E040E05EE30E9425
:10031000330C7B018C010E948F120E94650E1B0121
:100320002C01B101882777FD8095982F0E94070E38
:100330009B01AC01C801B7010E94D50B20E030E061
:100340004AE754E40E94330C0E948F123B014C0197
:10035000CF5FDE4F688179818A819B81C150D14016
:100360000E948F120E94650E5B016C01B501882707
:1003700077FD8095982F0E94070E9B01AC01CF5FFF
:10038000DE4F688179818A819B81C150D1400E9472
:10039000D50B20E030E04AE754E40E94330C0E9481
:1003A0008F127B018C01C401B3010E94600A7F930C
:1003B0006F933F922F92C801B7010E94600A7F930A
:1003C0006F93BF92AF9229EB30E03F932F9381E080
:1003D0008F930E945304882499248DB79EB70B965F
:1003E0000FB6F8949EBF0FBE8DBF1ECF379A3598BB
:1003F00086B1887F866086B987B18F73806487B93C
:100400003D98339A10923E03789408953398379824
:10041000089596B1987F982B96B9089597B18295D3
:10042000880F880F807C9F73982B97B9089597B198
:100430008F71907E892B87B90895349A369A0895E2
:1004400086B18074089510923E0397B18F71907EAB
:10045000892B87B9349A369A3699FECF24B145B1A3
:10046000942F80E030E0282B392BC90108950E9499
:100470002302969587959695879508951F920F92DA
:100480000FB60F9211248F938FEF80933E038F91BD
:100490000F900FBE0F901F901895FC018FB7F89426
:1004A000718360835383428317821682158214827C
:1004B0008FBF0895CF93DF93DC014FB7F894EC0121
:1004C0008C819D81892B11F4E0E01CC0FD018681A7
:1004D0009781ED91FC911197E80FF91FE08101964A
:1004E000ED019F838E832A813B818217930720F041
:1004F000821B930B9F838E83ED018C819D810197DD
:100500009D838C834FBF8E2FDF91CF910895FC0187
:100510004FB7F8948481958168177907B0F4868184
:100520009781860F971F9783868322813381821755
:10053000930720F0821B930B978386838481958198
:10054000861B970B9583848302C0158214824FBF4C
:100550000895FC01CB012FB7F8942FBF2681378176
:1005600062817381820F931F0E943F110190F0817D
:10057000E02DE80FF91F808108951F93CF93DF933B
:10058000EC01162F4FB7F8942C813D816A817B8155
:100590002617370798F48E819F81820F931F0E9440
:1005A0003F11E881F981E80FF91F10838C819D814B
:1005B00001969D838C834FBF8FEF02C04FBF80E0B9
:1005C000DF91CF911F910895FC018FB7F8948FBFF1
:1005D0002281338184819581281B390BC9010895BB
:1005E000FC018FB7F894158214828FBF0895909301
:1005F00009028093080208951F93182F8A3031F45E
:10060000E0910802F09109028DE00995E09108025D
:10061000F0910902812F09951F910895CF93DF93DF
:10062000EC01009721F406C021960E94FC0288810B
:100630008823D1F7DF91CF910895EF92FF920F9326
:100640001F93CF93DF938C017A010097E9F020E0AC
:1006500030E02617370738F4F80181918F012F5FBA
:100660003F4F8823B1F7C0E0D0E00BC0F801808194
:10067000882319F00F5F1F4F01C080E20E94FC0227
:100680002196CE15DF0590F3DF91CF911F910F9149
:10069000FF90EF900895CF93DF93EC01009719F44A
:1006A00007C00E94FC02FE01219684918823C9F7AD
:1006B000DF91CF9108958AE00E94FC020895E82F0F
:1006C000F0E0EF70F070E153FF4FE4918E2F0E9445
:1006D000FC0208951F93182F82958F700E945F036C
:1006E000812F0E945F031F9108951F93182F892F58
:1006F0000E946A03812F0E946A031F910895EF925E
:10070000FF920F931F937B018C01C801AA27BB277F
:100710000E947503C7010E9475031F910F91FF90FE
:10072000EF9008952F923F924F925F926F927F9237
:100730008F929F92AF92BF92CF92DF92EF92FF92F1
:100740000F931F93DF93CF93CDB7DEB7A3970FB669
:10075000F894DEBF0FBECDBF4AA32BA337014801DB
:10076000442351F017FF08C0EE24FF248701E61848
:10077000F7080809190902C084017301262E262FE3
:10078000215090E03AA1311191E0291B29A318A230
:10079000A82EBB24A7FCB094CB2CDB2CC801B7013E
:1007A000A60195010E945311FB01EF70F070E15317
:1007B000FF4F64916F8FC801B701A60195010E9498
:1007C0005311C901DA017C018D019EE1492E512CA2
:1007D0004C0E5D1E39A025C0E114F1040105110580
:1007E000C9F0C801B701A60195010E945311FB0190
:1007F000EF70F070E153FF4F6491F2016083C80124
:10080000B701A60195010E945311C901DA017C01CB
:100810008D0103C02BA1F20120833A940894410872
:1008200051083320C9F6CE014F968C0139A1031B24
:1008300011098AA18823E1F097FE05C08DE2F80135
:1008400082938F0115C0C80101976114710481045E
:10085000910419F08C018BE202C08C0180E2F80156
:10086000808306C0F80181918F010E94FC022A94C6
:100870002220C1F7A3960FB6F894DEBF0FBECDBFFE
:10088000CF91DF911F910F91FF90EF90DF90CF906C
:10089000BF90AF909F908F907F906F905F904F90A0
:1008A0003F902F9008957F928F929F92AF92BF9228
:1008B000CF92DF92EF92FF920F931F93DF93CF932C
:1008C000CDB7DEB77888C988DA8853E1E52EF12CF8
:1008D000EC0EFD1E14C0882381F480E090E0CF91DF
:1008E000DF911F910F91FF90EF90DF90CF90BF901D
:1008F000AF909F908F907F9008950E94FC02960188
:100900002F5F3F4F772021F0F6016901849103C0EA
:10091000F601808169018532F1F62F5F3F4F772024
:1009200021F0F6016901849103C0F601808169011B
:10093000843629F0883781F08336F9F606C000E165
:1009400017E24AE0A42EB12C0CC0F701808122E00E
:1009500030E0E20EF31ED1CF00E010E130E1A32E33
:10096000B12C22E0822E912C8E0C9F1CF701E0808E
:10097000F1808436B1F4F7FE11C0F094E194F108EF
:10098000F3948DE20E94FC0209C0C8016AE070E0A5
:100990000E943F118B016230710518F0E016F106DC
:1009A000A0F3C701B8010E943F11862F0E945F0388
:1009B000C701B8010E943F117C01C801B5010E9426
:1009C0003F118B016115710561F7740198CF08958E
:1009D00080E090E0FC01EE0FFF1FE65FFD4F11820B
:1009E0001082019688309105A9F783B7887F8260CD
:1009F00083BF12BE87B7816087BF10923F031092FA
:100A0000400310924103109242038EB5887F8360A9
:100A10008EBD1DBC1CBC87B7846087BF85B5887F31
:100A2000846085BD14BC87B7806487BF109247037C
:100A3000109248031092490310924A037894089543
:100A400083B7887F826083BF12BE87B7816087BF0C
:100A500010923F0310924003109241031092420300
:100A600008958EB5887F83608EBD1DBC1CBC87B782
:100A7000846087BF089585B5887F846085BD14BC78
:100A800087B7806487BF1092470310924803109283
:100A9000490310924A03089593B7987F982B93BF08
:100AA00008959EB5987F982B9EBD089595B5987F23
:100AB000982B95BD089583B7E82FF0E0E770F070AC
:100AC000EE0FFF1FE052FF4F25913491C9010895A9
:100AD0008EB5E82FF0E0E770F070EE0FFF1FE052E8
:100AE000FF4F25913491C901089585B5E82FF0E0B5
:100AF000E770F070EE0FFF1FE451FF4F2591349126
:100B0000C9010895883040F4E82FF0E0EE0FFF1F90
:100B1000E65FFD4F718360830895883040F4E82FCD
:100B2000F0E0EE0FFF1FE65FFD4F11821082089587
:100B3000EF92FF920F931F93CF93DF93EC0112B7C5
:100B400010924303109244031092450310924603FF
:100B500083B7E82FF0E0E770F070EE0FFF1FE05270
:100B6000FF4F2591349140E050E060E072E18AE768
:100B700090E00E947511B901CA01693B2DE8720726
:100B800026E0820720E09207A0F437E2C131D307C4
:100B900080F49E0140E050E00E94201128EE33E0F6
:100BA00040E050E00E945311C901DA01BC01CD01BF
:100BB00021C028EE33E040E050E00E945311CA010A
:100BC000B9019E0140E050E00E94201113C08091C5
:100BD000430390914403A0914503B091460385B728
:100BE000837E85BF85B7806285BF889585B78F7DF9
:100BF00085BF08C09B01AC01210F311D411D511D56
:100C000079018A01209143033091440340914503C7
:100C10005091460382B790E0A0E0B0E0542F432FFC
:100C2000322F2227822B932BA42BB52B8E159F05B9
:100C3000A007B10760F2DF91CF911F910F91FF9054
:100C4000EF90089510923F031092400310924103D9
:100C500010924203089520913F0330914003409148
:100C6000410350914203B901CA010895109247030C
:100C7000109248031092490310924A03089520915C
:100C80004703309148034091490350914A03B90109
:100C9000CA010895893031F48FB582608FBD8FB558
:100CA0008E7F0AC08A3019F48FB5826002C08FB57A
:100CB0008D7F8FBD8FB581608FBD1BBC1ABC19BCE9
:100CC00018BC08952FB52E7F2FBD2FB522602FBDE4
:100CD0002EB528602EBD2EB520612EBD97BD86BDD8
:100CE0001BBC1ABC19BC18BC08958FB58D7F8FBD75
:100CF0008FB58E7F8FBD8FB58F778FBD8FB58F7B73
:100D00008FBD8FB58F7D8FBD8FB58F7E8FBD0895C1
:100D10008FB580688FBD8FB58F7B8FBD08958FB5E0
:100D200080628FBD8FB58F7E8FBD08958FB58F7711
:100D30008FBD8FB58F7B8FBD08958FB58F7D8FBD94
:100D40008FB58F7E8FBD08959BBD8ABD089599BDD7
:100D500088BD08951F920F920FB60F9211248F93A2
:100D60009F93AF93BF93EF93FF9380913F03909135
:100D70004003A0914103B09142030196A11DB11D12
:100D800080933F0390934003A0934103B0934203A9
:100D90008091430390914403A0914503B091460391
:100DA0000196A11DB11D8093430390934403A0932A
:100DB0004503B093460380910A0290910B02892B60
:100DC00029F0E0910A02F0910B020995FF91EF9151
:100DD000BF91AF919F918F910F900FBE0F901F9079
:100DE00018951F920F920FB60F9211248F939F9315
:100DF000EF93FF9380910C0290910D02892B29F0C3
:100E0000E0910C02F0910D020995FF91EF919F91F5
:100E10008F910F900FBE0F901F9018951F920F92F9
:100E20000FB60F9211248F939F93AF93BF93EF93BD
:100E3000FF938091470390914803A0914903B0919B
:100E40004A030196A11DB11D809347039093480367
:100E5000A0934903B0934A03809114029091150224
:100E6000892B29F0E0911402F09115020995FF9168
:100E7000EF91BF91AF919F918F910F900FBE0F9007
:100E80001F9018951F920F920FB60F9211248F93F7
:100E90009F93EF93FF938091180290911902892BF1
:100EA00029F0E0911802F09119020995FF91EF9154
:100EB0009F918F910F900FBE0F901F9018951F92CA
:100EC0000F920FB60F9211248F939F93EF93FF937E
:100ED00080910E0290910F02892B29F0E0910E0271
:100EE000F0910F020995FF91EF919F918F910F90D3
:100EF0000FBE0F901F9018951F920F920FB60F9272
:100F000011248F939F93EF93FF9380911002909100
:100F10001102892B29F0E0911002F091110209953C
:100F2000FF91EF919F918F910F900FBE0F901F90A7
:100F300018951F920F920FB60F9211248F939F93C3
:100F4000EF93FF938091120290911302892B29F065
:100F5000E0911202F09113020995FF91EF919F9198
:100F60008F910F900FBE0F901F9018951F920F92A8
:100F70000FB60F9211248F939F93EF93FF9380915D
:100F8000160290911702892B29F0E0911602F09138
:100F900017020995FF91EF919F918F910F900FBECE
:100FA0000F901F901895823040F4E82FF0E0EE0F7C
:100FB000FF1FE65CFC4F7183608308951F93182F19
:100FC0009A01AB01CA01B901605C7D4B804F9F4F14
:100FD000F3E0660F771F881F991FFA95D1F7E4E0B9
:100FE000220F331F441F551FEA95D1F70E9453115A
:100FF00021503040112329F020939900309398001C
:1010000003C029B9309390001F910895282F30E034
:10101000A3E0220F331FAA95E1F7235B3C4FC901E0
:101020000895282F30E0B3E0220F331FBA95E1F77F
:10103000215A3C4FC9010895E82F882339F0809147
:101040009B0085FFFCCF60939C0003C05D9BFECF9F
:101050006CB9F0E0E55BFC4F108208955D9BFECF1C
:101060008CB910924B030895982F80919B0085FFB7
:10107000FCCF90939C0010924C03089520E0E82F41
:10108000F0E083E0EE0FFF1F8A95E1F7EF5AFC4F87
:1010900080819181892B09F421E0822F0895CF93DB
:1010A000DF93882319F060919C0001C06CB1282F58
:1010B00030E0E901CC0FDD1FFE01E65CFC4F8081D2
:1010C0009181892B31F00190F081E02D862F0995D7
:1010D00014C093E0220F331F9A95E1F7C901835B97
:1010E0009C4F0E94BD02882341F4FE01E159FC4F50
:1010F00080819181019691838083DF91CF910895C2
:101100001F920F920FB60F9211248F9381E00E94CD
:101110004F088F910F900FBE0F901F9018951F9240
:101120000F920FB60F9211248F9380E00E944F0808
:101130008F910F900FBE0F901F9018958F929F92D6
:10114000AF92BF92CF92DF92EF92FF920F931F93D5
:10115000CF93DF93882EDB01E82EFF24F70113E005
:10116000EE0FFF1F1A95E1F7ED59FC4F20813181F9
:10117000240F351FF70173E0EE0FFF1F7A95E1F79B
:10118000EF59FC4F8081918128173907D0F541151F
:101190005105B9F19C90670163E0CC0CDD1C6A95A8
:1011A000E1F78FE593E0C80ED91E8D01C0E0D0E0D5
:1011B0005A010894A108B10806C0F8016081C6016F
:1011C0000E94BD0221960F5F1F4FCA15DB05A8F3D1
:1011D000F701E35AFC4F8FEF8083882039F080912C
:1011E0009B0085FFFCCF90929C0003C05D9BFECFCF
:1011F0009CB88BE493E0E80EF91EF70110828FEFA4
:1012000001C080E0DF91CF911F910F91FF90EF908F
:10121000DF90CF90BF90AF909F908F90089590E017
:1012200023E0880F991F2A95E1F7815A9C4F0E946D
:10123000BD020895682F87E693E00E94BD020895DD
:10124000682F8FE593E00E94BD020895CF93DF934E
:10125000282FA82FB0E0ED01C35ADC4F88818823E6
:10126000E1F0FD0133E0EE0FFF1F3A95E1F7ED5994
:10127000FC4F80819181892B79F0222339F087E618
:1012800093E00E945A0280939C000BC08FE593E08C
:101290000E945A028CB905C01882A55BBC4F8FEF23
:1012A0008C93DF91CF9108951F920F920FB60F92FA
:1012B00011248F9381E00E9426098F910F900FBE19
:1012C0000F901F9018951F920F920FB60F92112436
:1012D0008F9380E00E9426098F910F900FBE0F9090
:1012E0001F9018951F93CF93DF93182FC82FD0E02E
:1012F000FE01E35AFC4F8FEF8083CE0143E0880F5D
:10130000991F4A95E1F7815A9C4F0E945A02982FE3
:10131000112339F080919B0085FFFCCF90939C00B6
:1013200003C05D9BFECF9CB9C55BDC4F1882DF918B
:10133000CF911F910895CF93DF93EB01282F30E0D9
:10134000F90173E0EE0FFF1F7A95E1F7E15BFC4FC7
:1013500080819181892BC9F0F90163E0EE0FFF1FB5
:101360006A95E1F7EF5AFC4F80819181892B69F0F2
:1013700053E0220F331F5A95E1F7C901835B9C4F5D
:101380000E945A0288838FEF01C080E0DF91CF91E5
:101390000895DF93CF930F92CDB7DEB7BE016F5F95
:1013A0007F4F81E00E949B09882319F42FEF3FEFC4
:1013B00003C08981282F30E0C9010F90CF91DF91C0
:1013C0000895DF93CF930F92CDB7DEB7BE016F5F65
:1013D0007F4F80E00E949B09882319F42FEF3FEF95
:1013E00003C08981282F30E0C9010F90CF91DF9190
:1013F000089590E0E3E0880F991FEA95E1F7835B99
:101400009C4F0E94F002089540E850E06AEA72E0C2
:1014100085E593E00E944D0240E150E06AE273E00E
:1014200087E693E00E944D0208950E94040A1092FC
:101430003D0310923C0388ED80939A0040E855E20A
:1014400060E070E081E00E94DE078FEF80934C0344
:1014500010925E03109272031092710378940895B3
:1014600040E850E06AE172E08DE493E00E944D02B2
:1014700040E150E06AE972E08FE593E00E944D029E
:1014800008950E94300A10923B0310923A0388EDAF
:101490008AB940E855E260E070E080E00E94DE0733
:1014A0008FEF80934B0310925D03109270031092A4
:1014B0006F03789408950E94410A0E94150A0895C6
:1014C000EF92FF920F931F937B018C0120E030E09D
:1014D00040E05FE40E94D70D88238CF020E030E0EC
:1014E00040E05FE4C801B7010E94D50B0E94650E81
:1014F0009B01AC01205030404040504806C0C8011C
:10150000B7010E94650E9B01AC01B901CA011F9190
:101510000F91FF90EF900895A0E0B0E0E2E9FAE0CB
:101520000C949011DC012B01FA019C91923008F48B
:1015300036C1EB018881823008F430C1943061F407
:10154000843009F02CC1FD0191818981981709F43B
:1015500026C1A0E0B1E023C1843009F41FC182306C
:10156000A9F4923009F01BC19A01AD0188E0EA01AB
:101570000990AE01E90109929E018150C1F7E20193
:101580008981ED0199818923818306C1923009F413
:1015900005C1ED012A803B80EB018A819B81ED0131
:1015A000AC80BD80CE80DF80EB01EC80FD800E81C1
:1015B0001F819101281B390BB90137FF04C0662731
:1015C0007727621B730B603271050CF061C0121635
:1015D00013066CF537014801062E04C096948794D3
:1015E000779467940A94D2F721E030E040E050E02D
:1015F00004C0220F331F441F551F6A95D2F7215094
:101600003040404050402E213F214023512321159E
:1016100031054105510521F021E030E040E050E086
:1016200079018A01E628F728082919293CC0232BCB
:10163000D1F1260E371E35014601062E04C09694C0
:101640008794779467940A94D2F721E030E040E0E1
:1016500050E004C0220F331F441F551F6A95D2F774
:1016600021503040404050402A213B214C215D21F7
:10167000211531054105510521F021E030E040E020
:1016800050E059016A01A628B728C828D9280BC0FC
:10169000821593052CF01C01AA24BB24650103C00C
:1016A000EE24FF248701ED019981E20189819817D9
:1016B00009F445C0992339F0A80197012A193B097B
:1016C0004C095D0906C0A60195012E193F09400B82
:1016D000510B57FD08C01182338222822483358347
:1016E000468357831DC081E081833382228288270D
:1016F0009927DC01821B930BA40BB50B8483958384
:10170000A683B7830DC0220F331F441F551F2483A8
:1017100035834683578382819381019793838283A4
:101720002481358146815781DA01C9010197A109D8
:10173000B1098F5F9F4FAF4FBF4328F30BC0918319
:1017400033822282EA0CFB1C0C1D1D1DE482F582F3
:101750000683178383E08083248135814681578106
:1017600057FF1AC0C901AA2797FDA095BA2F81700B
:101770009070A070B0705695479537952795822B3D
:10178000932BA42BB52B84839583A683B783828167
:101790009381019693838283DF0101C0D201CD0141
:1017A000CDB7DEB7E2E10C94AC11A0E2B0E0EBED16
:1017B000FBE00C949C1169837A838B839C832D833B
:1017C0003E834F835887E9E0EE2EF12CEC0EFD1E90
:1017D000B701CE0101960E9456108E010F5E1F4F79
:1017E000B801CE0105960E9456108A8991E089279A
:1017F0008A8BAE01475E5F4FB801C7010E948C0A19
:101800000E94810FA096E6E00C94B811A0E2B0E02F
:10181000ECE0FCE00C949C1169837A838B839C83BD
:101820002D833E834F835887F9E0EF2EF12CEC0E89
:10183000FD1EB701CE0101960E9456108E010F5E6B
:101840001F4FB801CE0105960E945610AE01475EAB
:101850005F4FB801C7010E948C0A0E94810FA096B9
:10186000E6E00C94B811A0E2B0E0E9E3FCE00C94EF
:10187000901169837A838B839C832D833E834F836E
:101880005887BE01675F7F4FCE0101960E945610B8
:10189000BE016F5E7F4FCE0105960E94561099855E
:1018A000923088F089898230C8F0943019F48230FF
:1018B00051F404C0843029F4923081F480E091E046
:1018C000C6C0923049F420E09A858A89981321E0B5
:1018D0002A87CE010996BBC0823049F420E09A8560
:1018E0008A89981321E02A8BCE014196B0C02D84BD
:1018F0003E844F8458886D887E888F88988CEE242B
:10190000FF248701AA24BB24650140E050E060E089
:1019100070E0E0E0F0E0C10181709070892BE9F0A7
:10192000E60CF71C081D191D9A01AB012A0D3B1D81
:101930004C1D5D1D80E090E0A0E0B0E0E614F704EF
:101940000805190520F481E090E0A0E0B0E0BA01BC
:10195000A901480F591F6A1F7B1FAA0CBB1CCC1C76
:10196000DD1C97FE08C081E090E0A0E0B0E0A82A6E
:10197000B92ACA2ADB2A3196E032F10549F0660C11
:10198000771C881C991C5694479437942794C3CF8E
:10199000FA85EA892B893C898B859C85280F391F1C
:1019A0002E5F3F4F17C0CA0181709070892B61F084
:1019B00016950795F794E79480E090E0A0E0B0E8F2
:1019C000E82AF92A0A2B1B2B769567955795479598
:1019D0002F5F3F4F77FDE7CF0CC0440F551F661FA9
:1019E000771F17FD4160EE0CFF1C001F111F2150D7
:1019F0003040403090E0590790E0690790E4790763
:101A000060F32B8F3C8FDB01CA018F779070A07041
:101A1000B07080349105A105B10561F447FD0AC09D
:101A2000E114F1040105110529F0405C5F4F6F4F8F
:101A30007F4F40781A8EFE1711F081E08A8F4D8F0C
:101A40005E8F6F8F78A383E0898FCE0149960E94C5
:101A5000810FA096E2E10C94AC11A8E1B0E0E3E3C1
:101A6000FDE00C94981169837A838B839C832D838A
:101A70003E834F835887B9E0EB2EF12CEC0EFD1E10
:101A8000B701CE0101960E9456108E010F5E1F4FC6
:101A9000B801CE0105960E9456102985223008F41F
:101AA0007CC03989323010F4B8017AC08A859A89AD
:101AB00089278A87243011F0223031F4231709F066
:101AC0006CC060E071E06CC0343039F41D861E8655
:101AD0001F86188A1C861B8604C0323021F484E0DD
:101AE0008987B7015DC02B853C858B899C89281B24
:101AF000390B3C872B87ED84FE840F851889AD88D0
:101B0000BE88CF88D88CEA14FB040C051D0540F470
:101B1000EE0CFF1C001F111F215030403C872B870B
:101B200020E030E040E050E080E090E0A0E0B0E471
:101B30006FE170E0EA14FB040C051D0540F0282B52
:101B4000392B4A2B5B2BEA18FB080C091D09B695AB
:101B5000A79597958795EE0CFF1C001F111F6150EC
:101B6000704041F7DA01C9018F779070A070B070B2
:101B700080349105A105B10561F427FD0AC0E11487
:101B8000F1040105110529F0205C3F4F4F4F5F4FD5
:101B900020782D873E874F87588BBE01675F7F4F28
:101BA000CB010E94810F6896EAE00C94B411A8E181
:101BB000B0E0EDEDFDE00C949C1169837A838B839A
:101BC0009C832D833E834F83588789E0E82EF12C38
:101BD000EC0EFD1EB701CE0101960E9456108E013B
:101BE0000F5E1F4FB801CE0105960E9456108985E1
:101BF000823040F08989823028F0B801C7010E9404
:101C0000C61001C08FEF6896E6E00C94B811A8E00A
:101C1000B0E0EDE0FEE00C9499119B01AC0183E093
:101C20008983DA01C9018827B7FD83959927AA27F7
:101C3000BB27B82E211531054105510519F482E065
:101C400089833AC08823A9F0203080E0380780E0FB
:101C5000480780E8580729F460E070E080E09FECD6
:101C600030C0EE24FF248701E21AF30A040B150B9F
:101C700002C079018A018EE1C82ED12CDC82CB8290
:101C8000ED82FE820F831887C801B7010E94320FD0
:101C900001971816190684F4082E04C0EE0CFF1CD8
:101CA000001F111F0A94D2F7ED82FE820F8318875E
:101CB000C81AD90ADC82CB82BA82CE0101960E9470
:101CC000810F2896E9E00C94B511ACE0B0E0EBE6AA
:101CD000FEE00C94A01169837A838B839C83BE0100
:101CE0006B5F7F4FCE0101960E9456108D8182302E
:101CF00061F1823050F1843021F48E81882351F1DA
:101D00002EC02F81388537FD20C06E812F313105DF
:101D10001CF06623F9F023C08EE190E0821B930B48
:101D200029853A854B855C8504C05695479537953E
:101D300027958A95D2F76623B1F050954095309556
:101D400021953F4F4F4F5F4F0EC020E030E040E005
:101D500050E009C02FEF3FEF4FEF5FE704C020E0F6
:101D600030E040E050E8B901CA012C96E2E00C9462
:101D7000BC11A8E0B0E0EFEBFEE00C949A117B01FF
:101D80008C01611571058105910519F482E0898343
:101D900060C083E089838EE1C82ED12CDC82CB82A7
:101DA000ED82FE820F831887C801B7010E94320FAF
:101DB000BC016150704077FF39C0EE27FF27E61B5A
:101DC000F70B20E030E040E050E081E090E0A0E060
:101DD000B0E00E2E04C0880F991FAA1FBB1F0A94E3
:101DE000D2F70197A109B1098E219F21A023B12328
:101DF0000097A105B10521F021E030E040E050E07E
:101E000004C016950795F794E794EA95D2F72E2922
:101E10003F29402B512B2D833E834F8358878EE1E2
:101E200090E0861B970B9C838B8313C06115710513
:101E300081F0062E04C0EE0CFF1C001F111F0A9437
:101E4000D2F7ED82FE820F831887C61AD70ADC828A
:101E5000CB821A82CE0101960E94810F2896E8E07B
:101E60000C94B611EF92FF920F931F937B018C019C
:101E700080E0E81680E0F80681E0080780E01807B7
:101E800088F48FEFE816F1040105110531F028F010
:101E900088E090E0A0E0B0E017C080E090E0A0E033
:101EA000B0E012C080E0E81680E0F80680E00807A5
:101EB00081E0180728F088E190E0A0E0B0E004C0DD
:101EC00080E190E0A0E0B0E020E230E040E050E0CF
:101ED000281B390B4A0B5B0B04C016950795F7942A
:101EE000E7948A95D2F7F701E85FFE4F8081281BBF
:101EF000310941095109C9011F910F91FF90EF90DC
:101F00000895DF92EF92FF920F931F93FC01E480FC
:101F1000F58006811781D1808081823048F480E08D
:101F200090E0A0E1B0E0E82AF92A0A2B1B2BA5C01B
:101F3000843009F49FC0823021F4EE24FF2487010D
:101F400005C0E114F1040105110519F4E0E0F0E029
:101F500096C0628173819FEF623879070CF05BC095
:101F600022E83FEF261B370B2A3131052CF020E009
:101F700030E040E050E02AC0B801A701022E04C0C2
:101F800076956795579547950A94D2F781E090E04A
:101F9000A0E0B0E004C0880F991FAA1FBB1F2A95BC
:101FA000D2F70197A109B1098E219F21A023B12366
:101FB0000097A105B10521F081E090E0A0E0B0E03C
:101FC0009A01AB01282B392B4A2B5B2BDA01C90173
:101FD0008F779070A070B07080349105A105B10525
:101FE00039F427FF09C0205C3F4F4F4F5F4F04C0BB
:101FF000215C3F4F4F4F5F4FE0E0F0E02030A0E02A
:102000003A07A0E04A07A0E45A0710F0E1E0F0E048
:1020100079018A0127C06038710564F5FB01E15838
:10202000FF4FD801C7018F779070A070B0708034D7
:102030009105A105B10539F4E7FE0DC080E490E0FB
:10204000A0E0B0E004C08FE390E0A0E0B0E0E80ED4
:10205000F91E0A1F1B1F17FF05C016950795F79459
:10206000E794319687E016950795F794E7948A955B
:10207000D1F705C0EE24FF248701EFEFF0E06E2FCB
:10208000679566276795902F9F77D794DD24D7941F
:102090008E2F8695492F462B582F5D29B701CA01EF
:1020A0001F910F91FF90EF90DF900895FC01DB01ED
:1020B000408151812281622F6F7770E0221F222799
:1020C000221F9381892F880F822B282F30E0991FA0
:1020D0009927991FFD0191832115310581F541153E
:1020E00051056105710511F482E032C082E89FEF6D
:1020F000FD01938382839A01AB0167E0220F331FB6
:10210000441F551F6A95D1F783E08C930AC0220FB4
:10211000331F441F551FFD018281938101979383D3
:1021200082832030F0E03F07F0E04F07F0E45F07E4
:1021300070F3FD01248335834683578308952F3F31
:10214000310581F4411551056105710519F484E0EB
:102150008C93089564FF03C081E08C9301C01C92AE
:10216000FD010FC02F573040FD013383228383E0F0
:102170008C9387E0440F551F661F771F8A95D1F710
:102180007064448355836683778308951F93CF9348
:10219000DF93DC01FB019C91923008F444C0808104
:1021A000823008F440C0943051F4ED01198184303C
:1021B00081F58181682F70E0611B71093CC084301A
:1021C00021F0923031F48230A1F18181882371F1C4
:1021D0002AC0ED0119818230E1F081811817C9F41C
:1021E000ED012A813B8182819381821793078CF0D4
:1021F00028173907B4F0ED018C819D81AE81BF8134
:102200002481358146815781281739074A075B07A2
:1022100018F4112341F00AC082179307A407B507E9
:1022200040F4112319F061E070E005C06FEF7FEF1B
:1022300002C060E070E0CB01DF91CF911F91089563
:10224000629FD001739FF001829FE00DF11D649F9A
:10225000E00DF11D929FF00D839FF00D749FF00D26
:10226000659FF00D9927729FB00DE11DF91F639FC7
:10227000B00DE11DF91FBD01CF0111240895AA1B66
:10228000BB1B51E107C0AA1FBB1FA617B70710F061
:10229000A61BB70B881F991F5A95A9F78095909593
:1022A000BC01CD010895A1E21A2EAA1BBB1BFD01A2
:1022B0000DC0AA1FBB1FEE1FFF1FA217B307E40725
:1022C000F50720F0A21BB30BE40BF50B661F771F7D
:1022D000881F991F1A9469F760957095809590955D
:1022E0009B01AC01BD01CF01089597FB092E052686
:1022F0000ED057FD04D0D7DF0AD0001C38F450951B
:102300004095309521953F4F4F4F5F4F0895F6F719
:1023100090958095709561957F4F8F4F9F4F089551
:102320002F923F924F925F926F927F928F929F92E5
:10233000AF92BF92CF92DF92EF92FF920F931F93D3
:10234000CF93DF93CDB7DEB7CA1BDB0B0FB6F89484
:10235000DEBF0FBECDBF09942A88398848885F84C4
:102360006E847D848C849B84AA84B984C884DF8035
:10237000EE80FD800C811B81AA81B981CE0FD11D19
:102380000FB6F894DEBF0FBECDBFED01089533D177
:1023900058F080E891E009F49EEF34D128F040E84D
:1023A00051E059F45EEF09C0FEC07DC1E92FE0782D
:1023B00041D168F3092E052AC1F3261737074807CC
:1023C000590738F00E2E07F8E02569F0E025E064A3
:1023D0000AC0EF6307F8009407FADB01B9019D0119
:1023E000DC01CA01AD01EF9341D013D10AD05F9156
:1023F000552331F02BED3FE049E450FD49EC06CA8E
:102400000895DF93DD27B92FBF7740E85FE3161605
:10241000170648075B0710F4D92F4CD19F938F9371
:102420007F936F93FDD1ECE8F0E0C0D0F2D02F9114
:102430003F914F915F914FD1DD2349F09058A2EA2F
:102440002AED3FE049EC5FE3D0785D27F9D1DF91D9
:10245000E0C0D8D040F0CFD030F021F45F3F19F089
:1024600071C0511121C19FC0E5D098F39923C9F3E0
:102470005523B1F3951B550BBB27AA27621773078A
:10248000840738F09F5F5F4F220F331F441FAA1F3E
:10249000A9F333D00E2E3AF0E0E830D091505040FE
:1024A000E695001CCAF729D0FE2F27D0660F771FAC
:1024B000881FBB1F261737074807AB07B0E809F08E
:1024C000BB0B802DBF01FF2793585F4F2AF09E3F23
:1024D000510568F037C0E8C05F3FECF3983EDCF38D
:1024E000869577956795B795F7959F5FC9F7880F9C
:1024F000911D9695879597F90895E1E0660F771FEE
:10250000881FBB1F621773078407BA0720F0621B7E
:10251000730B840BBA0BEE1F88F7E0950895ACD0CF
:1025200080F09F3740F491110EF0BEC060E070E083
:1025300080E89FEB089526F41B16611D711D811D17
:1025400007C021C097F99F6780E870E060E00895B8
:10255000882371F4772321F09850872B762F07C0BA
:10256000662311F499270DC09051862B70E060E02E
:102570002AF09A95660F771F881FDAF7880F9695CD
:10258000879597F908959F3F49F0915028F48695D3
:1025900077956795B7959F5F80389F4F880F969581
:1025A000879597F908959FEF80EC0895DF93CF9377
:1025B0001F930F93FF92EF92DF927B018C0168943F
:1025C00005C0DA2EEF0187D0FE01E894A591259190
:1025D000359145915591AEF3EF0132D1FE0197014E
:1025E000A801DA9479F7DF90EF90FF900F911F9197
:1025F000CF91DF91089500240A9416161706180645
:102600000906089500240A941216130614060506F6
:102610000895092E0394000C11F4882352F0BB0F87
:1026200040F4BF2B11F460FF04C06F5F7F4F8F4FEA
:102630009F4F089557FD9058440F551F59F05F3F25
:1026400071F04795880F97FB991F61F09F3F79F0D4
:1026500087950895121613061406551FF2CF469556
:10266000F1DF08C0161617061806991FF1CF8695D8
:102670007105610508940895E5DFA0F0BEE7B9177C
:1026800088F4BB279F3860F41616B11D672F782F8A
:102690008827985FF7CF869577956795B11D9395B5
:1026A0009639C8F30895E894BB2766277727CB01AE
:1026B00097F908959B01AC0160E070E080E89FE32A
:1026C000CCC999DF28F09EDF18F0952309F03ACFA6
:1026D0006ACF1124E9CFAEDFA0F3959FD1F3950F18
:1026E00050E0551F629FF001729FBB27F00DB11D96
:1026F000639FAA27F00DB11DAA1F649F6627B00D26
:10270000A11D661F829F2227B00DA11D621F739F0E
:10271000B00DA11D621F839FA00D611D221F749F1C
:102720003327A00D611D231F849F600D211D822F63
:10273000762F6A2F11249F5750408AF0E1F08823AA
:102740004AF0EE0FFF1FBB1F661F771F881F9150B7
:102750005040A9F79E3F510570F0F4CEA5CF5F3FE2
:10276000ECF3983EDCF3869577956795B795F795EA
:10277000E7959F5FC1F7FE2B880F911D9695879572
:1027800097F9089511F40EF40ECFFDCE5BDFD0F370
:102790009923D9F3CEF39F57550B87FFA4D05695B5
:1027A0009795B0E020F4660F771F881FBB1F1F931B
:1027B0000F9300249001A0018001F001A0E80E0F0A
:1027C0001F1F0A1E511D601B710B8009B50B48F4B9
:1027D000600F711F801DB51F0E1B1F0B0A0A5109C8
:1027E00007C02E0F3F1F4A1F0E0F1F1F0A1E511D2D
:1027F000660F771F881FBB1FA695F795E795F8F61C
:102800000617170708065B07211D311D411D0F9193
:102810001F91B901842F9158880F96958795089537
:102820009B01AC0120C8E7DE30F0ECDE20F031F493
:102830009F3F11F41EF4B7CE0EF4E095E7FB82CE75
:10284000E92FF8DE80F3BA1762077307840795074C
:1028500018F071F49EF527CF0EF4E0950B2EBA2FE9
:10286000A02D0B01B90190010C01CA01A001112496
:10287000FF27591B99F0593F50F4503E68F11A1642
:10288000F040A22F232F342F4427585FF3CF4695D3
:1028900037952795A795F0405395C9F77EF41F16F5
:1028A000BA0B620B730B840BBAF09150A1F0FF0FBF
:1028B000BB1F661F771F881FC2F70EC0BA0F621FAB
:1028C000731F841F48F4879577956795B795F7959B
:1028D0009E3F08F0B3CF9395880F08F09927EE0F2D
:1028E00097958795089591505040660F771F881FE0
:0828F000D2F70895F894FFCF20
:1028F80000000000000000000001020203030303BF
:102908000404040404040404050505050505050577
:102918000505050505050505060606060606060657
:10292800060606060606060606060606060606063F
:102938000606060606060606070707070707070727
:10294800070707070707070707070707070707070F
:1029580007070707070707070707070707070707FF
:1029680007070707070707070707070707070707EF
:1029780007070707070707070808080808080808D7
:1029880008080808080808080808080808080808BF
:1029980008080808080808080808080808080808AF
:1029A800080808080808080808080808080808089F
:1029B800080808080808080808080808080808088F
:1029C800080808080808080808080808080808087F
:1029D800080808080808080808080808080808086F
:1029E800080808080808080808080808080808085F
:0829F800080808080808080897
:00000001FF
